LX51 CODE BANKING LINKER/LOCATOR V05.01.29                                     12/09/08  00:57:43
WIN32 LX51 CODE BANKING LINKER/LOCATOR V05.01.29,  INVOKED BY:
LX51 c:\test\ir_control\ir_remote_led.obj , c:\test\ir_control\ir_control.DTP TO(c:\test\ir_contr&
ol\ir_control.AOF) PR(c:\test\ir_control\ir_control.m51) XSIZE(65536) CSIZE(65536) RS(256) RSI(12&
8) IX MAP 


MEMORY MODEL: SMALL WITHOUT ANY FLOATING POINT ARITHMETIC


INPUT MODULES INCLUDED
  C:\TEST\IR_CONTROL\IR_REMOTE_LED.OBJ(IR_REMOTE_LED)
  C:\TEST\IR_CONTROL\IR_CONTROL.DTP(_WKRDTP_)
  c:\RIDE\Lib\RC51S.LIB(C3S)
  c:\RIDE\Lib\RC51S.LIB(HPD)
  c:\RIDE\Lib\RC51S.LIB(_C_IDATALEN)


LINK MAP OF MODULE: C:\TEST\IR_CONTROL\IR_CONTROL.AOF (IR_CONTROL)

    TYPE     BASE       LENGTH    RELOCATION     SEGMENT NAME
    ----     ----       ------    ----------     ------------

    * * * * * * *   DATA/IDATA    M E M O R Y   * * * * * * *
    REG      0000H      0008H     ABSOLUTE       "REG BANK 0"
    DATA     0008H      000AH     UNIT           ?DT?IR_REMOTE_LED
    DATA     0012H      0001H     OVERLAID UNIT  _DGROUP02_
             0012H      0001H     -------------  ?DT?init_system?IR_REMOTE_LED
    IDATA    0013H      0001H     * * STACK * *  _STACK

    * * * * * * *   CODE          M E M O R Y   * * * * * * *
    CODE     0000H      0003H     ABSOLUTE       
    CODE     0003H      0003H     ABSOLUTE       
             0006H      0005H                    *** GAP ***
    CODE     000BH      0003H     ABSOLUTE       
    CODE     000EH      000FH     UNIT           ?PR?C51_STARTUP?
    CODE     001DH      001CH     UNIT           ?PR?_delay?IR_REMOTE_LED
    CODE     0039H      000BH     UNIT           ?PR?Timer0_int?IR_REMOTE_LED
    CODE     0044H      00A4H     UNIT           ?PR?EX0_int?IR_REMOTE_LED
    CODE     00E8H      003CH     UNIT           ?PR?init_system?IR_REMOTE_LED
    CODE     0124H      01AFH     UNIT           ?PR?main?IR_REMOTE_LED

EXECUTABLE SUMMARY:
-------------------
    Total INTERNAL RAM storage requirement:  0013H (19)
    Total EXTERNAL RAM storage requirement:  0000H (0)
    Total     CODE     storage requirement:  02CEH (718)
Note:  Summary does not include dynamic stack requirements


REFERENCE MAP OF MODULE: C:\TEST\IR_CONTROL\IR_CONTROL.AOF (IR_CONTROL)

SEGMENT                           BI_GROUP            DT_GROUP             ID_GROUP             XD_GROUP
  +--> CALLED SEGMENT          START    LENGTH     START    LENGTH     START    LENGTH     START    LENGTH
--------------------------------------------------------------------------------------

?PR?Timer0_int?IR_REMOTE_LED   ---------------     ---------------     ---------------     ---------------

?PR?EX0_int?IR_REMOTE_LED      ---------------     ---------------     ---------------     ---------------

?PR?main?IR_REMOTE_LED         ---------------     ---------------     ---------------     ---------------
  +--> ?PR?init_system?IR_REMOTE_LED
  +--> ?PR?_delay?IR_REMOTE_LED

?PR?init_system?IR_REMOTE_LED  ---------------     0012H    0001H     ---------------     ---------------
  +--> ?PR?_delay?IR_REMOTE_LED

?PR?_delay?IR_REMOTE_LED       ---------------     ---------------     ---------------     ---------------

SYMBOL TABLE FOR C:\TEST\IR_CONTROL\IR_CONTROL.AOF(IR_REMOTE_LED)
------------------------------------------------------------------

    VALUE              TYPE               NAME
    -----              ----               ----

	-------            MODULE             ir_remote_led
	C:0000H            SYMBOL             _ICE_DUMMY_
	C:0124H            PUBLIC             main
	C:00E8H            PUBLIC             init_system
	C:0044H            PUBLIC             EX0_int
	C:0039H            PUBLIC             Timer0_int
	C:001DH            PUBLIC             _delay
	D:0011H            PUBLIC             disp_led
	D:0010H            PUBLIC             ir_rx_temp
	D:000FH            PUBLIC             ir_rx_flag
	D:000EH            PUBLIC             ir_bit_cnt
	D:000DH            PUBLIC             ir_timer_cnt
	D:000CH            PUBLIC             ir_state
	D:0008H            PUBLIC             ir_rx_data
	B:00A0H            SYMBOL             BUZZ
	B:0098H            SYMBOL             RI
	B:0099H            SYMBOL             TI
	B:009AH            SYMBOL             RB8
	B:009BH            SYMBOL             TB8
	B:009CH            SYMBOL             REN
	B:009DH            SYMBOL             SM2
	B:009EH            SYMBOL             SM1
	B:009FH            SYMBOL             SM0
	B:00B0H            SYMBOL             RXD
	B:00B1H            SYMBOL             TXD
	B:00B2H            SYMBOL             INT0
	B:00B3H            SYMBOL             INT1
	B:00B4H            SYMBOL             T0
	B:00B5H            SYMBOL             T1
	B:00B6H            SYMBOL             WR
	B:00B7H            SYMBOL             RD
	B:00B8H            SYMBOL             PX0
	B:00B9H            SYMBOL             PT0
	B:00BAH            SYMBOL             PX1
	B:00BBH            SYMBOL             PT1
	B:00BCH            SYMBOL             PS
	B:00A8H            SYMBOL             EX0
	B:00A9H            SYMBOL             ET0
	B:00AAH            SYMBOL             EX1
	B:00ABH            SYMBOL             ET1
	B:00ACH            SYMBOL             ES
	B:00AFH            SYMBOL             EA
	B:0088H            SYMBOL             IT0
	B:0089H            SYMBOL             IE0
	B:008AH            SYMBOL             IT1
	B:008BH            SYMBOL             IE1
	B:008CH            SYMBOL             TR0
	B:008DH            SYMBOL             TF0
	B:008EH            SYMBOL             TR1
	B:008FH            SYMBOL             TF1
	B:00D0H            SYMBOL             P
	B:00D2H            SYMBOL             OV
	B:00D3H            SYMBOL             RS0
	B:00D4H            SYMBOL             RS1
	B:00D5H            SYMBOL             F0
	B:00D6H            SYMBOL             AC
	B:00D7H            SYMBOL             CY
	D:0099H            SYMBOL             SBUF
	D:0098H            SYMBOL             SCON
	D:00B8H            SYMBOL             IP
	D:00A8H            SYMBOL             IE
	D:008DH            SYMBOL             TH1
	D:008CH            SYMBOL             TH0
	D:008BH            SYMBOL             TL1
	D:008AH            SYMBOL             TL0
	D:0089H            SYMBOL             TMOD
	D:0088H            SYMBOL             TCON
	D:0087H            SYMBOL             PCON
	D:0083H            SYMBOL             DPH
	D:0082H            SYMBOL             DPL
	D:0081H            SYMBOL             SP
	D:00F0H            SYMBOL             B
	D:00E0H            SYMBOL             ACC
	D:00D0H            SYMBOL             PSW
	D:00B0H            SYMBOL             P3
	D:00A0H            SYMBOL             P2
	D:0090H            SYMBOL             P1
	D:0080H            SYMBOL             P0
	-------            PROC               _delay
	C:001DH            LINE#              22
	C:001DH            LINE#              22
	C:001DH            LINE#              26
	C:002AH            LINE#              27
	C:0038H            LINE#              29
	C:0038H            LINE#              29
	-------            ENDPROC            _delay
	-------            PROC               Timer0_int
	C:0039H            LINE#              32
	C:003DH            LINE#              32
	C:003DH            LINE#              34
	C:0043H            LINE#              35
	C:0043H            LINE#              35
	-------            ENDPROC            Timer0_int
	-------            PROC               EX0_int
	C:0044H            LINE#              40
	C:0052H            LINE#              40
	C:0052H            LINE#              42
	C:0054H            LINE#              44
	C:0060H            LINE#              46
	C:0063H            LINE#              47
	C:0065H            LINE#              51
	C:0071H            LINE#              52
	C:0074H            LINE#              54
	C:0077H            LINE#              55
	C:0079H            LINE#              56
	C:007BH            LINE#              60
	C:0089H            LINE#              64
	C:0095H            LINE#              65
	C:009AH            LINE#              68
	C:009DH            LINE#              69
	C:009FH            LINE#              72
	C:00A1H            LINE#              73
	C:00ABH            LINE#              74
	C:00B6H            LINE#              75
	C:00B9H            LINE#              77
	C:00C0H            LINE#              78
	C:00C3H            LINE#              79
	C:00C5H            LINE#              80
	C:00C8H            LINE#              83
	C:00CEH            LINE#              89
	C:00D1H            LINE#              91
	C:00D7H            LINE#              93
	C:00E7H            LINE#              94
	C:00E7H            LINE#              94
	-------            ENDPROC            EX0_int
	-------            PROC               init_system
	D:0012H            SYMBOL             l_cnt
	C:00E8H            LINE#              97
	C:00E8H            LINE#              97
	C:00E8H            LINE#              101
	C:00EAH            LINE#              102
	C:00EDH            LINE#              105
	C:00EFH            LINE#              106
	C:00F1H            LINE#              107
	C:00F3H            LINE#              111
	C:00F5H            LINE#              112
	C:00F8H            LINE#              113
	C:00FFH            LINE#              114
	C:0102H            LINE#              115
	C:0109H            LINE#              111
	C:0110H            LINE#              119
	C:0113H            LINE#              121
	C:0119H            LINE#              123
	C:011BH            LINE#              124
	C:011DH            LINE#              125
	C:011FH            LINE#              126
	C:0121H            LINE#              127
	C:0123H            LINE#              128
	C:0123H            LINE#              128
	-------            ENDPROC            init_system
	-------            PROC               main
	C:0124H            LINE#              130
	C:0124H            LINE#              130
	C:0124H            LINE#              132
	C:0127H            LINE#              136
	C:012AH            LINE#              138
	C:012FH            LINE#              139
	C:0131H            LINE#              141
	C:0133H            LINE#              142
	C:0136H            LINE#              145
	C:017EH            LINE#              149
	C:0181H            LINE#              150
	C:0188H            LINE#              151
	C:018BH            LINE#              152
	C:018EH            LINE#              156
	C:0191H            LINE#              157
	C:0198H            LINE#              158
	C:019BH            LINE#              159
	C:01A2H            LINE#              160
	C:01A5H            LINE#              161
	C:01ACH            LINE#              162
	C:01AFH            LINE#              163
	C:01B6H            LINE#              164
	C:01B9H            LINE#              165
	C:01C0H            LINE#              166
	C:01C3H            LINE#              167
	C:01CAH            LINE#              168
	C:01CDH            LINE#              169
	C:01D4H            LINE#              170
	C:01D7H            LINE#              171
	C:01DEH            LINE#              172
	C:01E1H            LINE#              173
	C:01E8H            LINE#              174
	C:01EBH            LINE#              175
	C:01F2H            LINE#              176
	C:01F5H            LINE#              180
	C:01F8H            LINE#              181
	C:01FFH            LINE#              182
	C:0202H            LINE#              183
	C:0209H            LINE#              184
	C:020CH            LINE#              185
	C:0213H            LINE#              186
	C:0216H            LINE#              187
	C:021DH            LINE#              188
	C:0220H            LINE#              189
	C:0227H            LINE#              190
	C:022AH            LINE#              191
	C:0231H            LINE#              192
	C:0234H            LINE#              193
	C:023BH            LINE#              194
	C:023EH            LINE#              195
	C:0245H            LINE#              196
	C:0248H            LINE#              197
	C:024FH            LINE#              198
	C:0252H            LINE#              199
	C:0259H            LINE#              200
	C:025BH            LINE#              204
	C:025EH            LINE#              205
	C:0265H            LINE#              206
	C:0268H            LINE#              207
	C:026AH            LINE#              211
	C:026DH            LINE#              212
	C:0274H            LINE#              213
	C:0277H            LINE#              214
	C:0279H            LINE#              218
	C:027CH            LINE#              219
	C:0283H            LINE#              220
	C:0286H            LINE#              221
	C:0288H            LINE#              225
	C:028BH            LINE#              226
	C:0292H            LINE#              227
	C:0295H            LINE#              228
	C:0297H            LINE#              232
	C:029AH            LINE#              233
	C:02A1H            LINE#              234
	C:02A4H            LINE#              235
	C:02A6H            LINE#              239
	C:02A9H            LINE#              240
	C:02B0H            LINE#              241
	C:02B3H            LINE#              242
	C:02B5H            LINE#              246
	C:02B8H            LINE#              247
	C:02BFH            LINE#              248
	C:02C2H            LINE#              254
	C:02C5H            LINE#              256
	C:02CCH            LINE#              257
	C:02CEH            LINE#              258
	C:02D0H            LINE#              261
	-------            ENDPROC            main
	-------            ENDMOD             ir_remote_led
	N:00E8H            PUBLIC             TIM1_INIT
	N:0010H            PUBLIC             SIZEBUFPRINTF
	N:0100H            PUBLIC             XSTACKLEN
	N:0001H            PUBLIC             _LINKERSYMB_DUMMY_
	C:000EH            PUBLIC             ?C_START3
	D:00A0H            PUBLIC             HPD_ADDR
	N:007FH            PUBLIC             IDATALEN
	N:00FFH            PUBLIC             _INITP2?

LINK/LOCATE RUN COMPLETE,  NO ERROR FOUND.

